:020000020000FC
:080000000C94CE010C94CC001D
:040014000C944B01FC
:040034000C948A019D
:040040000C94F80024
:040048000C946E0C9A
:100050000C943D0CBF93AF93A8E8B1E016E02D914E
:100060003D91232B31F016961A95C9F7EF91FF9128
:1000700016C0ED93FD93ED920D93EF91FF910191D9
:100080000D9301910D9318973297ED93FC93E831FE
:1000900029F4F13019F40BA100640BA31197089512
:1000A0000A2F0B2B89F0ED91FD9114960D911D9166
:1000B00001931193EA3131F4F13021F40BA10F7B5C
:1000C0000BA3C6D7189701D00895FD92FD92FD921B
:1000D000FD92FD92FD92FD92FD92089507E0A8E841
:1000E000B1E0F3DF0A95E9F70895A8E8B1E026E06A
:1000F000BF93AF930D911D91012B21F012972F9378
:1001000009952F91AF91BF9118962A9589F7089577
:100110000D911D9112962D913C913F3F19F03A950A
:100120003C9389F0322F319533953E93222321F071
:10013000D801FD92FD920DC012972D913D91D801ED
:100140002D933D9306C01597FF93EF93A9DFEF9191
:10015000FF9108954A2F4B2B59F04D914E1741F4C2
:100160004D914F1729F40D931D9312960D931D93E6
:100170000895E8E8F0E0B9DF08955A9A0E94E40C87
:1001800002E01E8510FD03E00093690001D0089590
:10019000E89A0895E89808950F930FB70F93946025
:1001A0000F910FBF0F9118950F93F4BC05E005BD9B
:1001B0000F910895BF93AF93ADE7B0E0AF8FB8A3B1
:1001C000AF91BF910895FF8EF8A208950F93FF8E0F
:1001D000F8A201E005BB01E806BD01E000936E0056
:1001E0000F9108950F9300E000936E000F91089512
:1001F0000F9301E806BD78940FB70F931F93BF9339
:10020000AF93AF8DB8A10A2F0B2B51F01197AF8F81
:10021000B8A331F400910402002311F49860FCA209
:100220000DA1000F1E2D4F9B1127012B0DA3003890
:1002300049F40CA10E15A1F00BA108600BA3ECA2D0
:10024000B9DF0EC00F3721F00F3F51F413D008C0B3
:100250000CA1002329F09062FCA20BA1077F0BA345
:10026000AF91BF911F910F910FBF0F9118950CD0B7
:10027000ADDF0895B7DF01D0089510E810936D0049
:1002800014E010936800089510E010936D0010E0E2
:100290001093680008950F930FB71F930F93E7DF34
:1002A0000F911F910FBF0F91189504E000938100EB
:1002B0000AEF009385000AEE0093840022D008958F
:1002C000BF93AF93A8E0B7E0F894A9A3BAA378943A
:1002D000AF91BF910895BF93AF93A8E7B0E0F894B2
:1002E000A9A3BAA37894AF91BF910895F9A2FAA2F5
:1002F00008951F9309A11AA1012B09F00E2D1F913A
:10030000089501E000936F00F1DF089500E000938D
:100310006F0008950F930AEE009384000AEF009394
:10032000850078940FB71F930F93BF93AF93A9A144
:10033000BAA10A2F0B2B21F01197A9A3BAA301F49C
:100340000F81002329F00A9511F4906808850F8326
:1003500008890A9511F490640FE0088BAF91BF9162
:100360000F911F910FBF0F911895A89504B7077FA4
:1003700004BF0091600008610093600000270093B3
:1003800060000895F894A8950091600008610093BA
:1003900060000AE00093600078940895F894E5DF27
:1003A0002227E0E0F1E014E0002721930A95E9F725
:1003B0001A95D1F7C0ECD1E0FF24EE24E3949927FD
:1003C000882499240FEF0DA308AB02E30EA30FE4DA
:1003D0000FA3E6E3FBE1E0930001F0930101E6ECFB
:1003E000FCE1E0930102F0930202E0930401F09338
:1003F0000501ECEAFAE2E0933401F09335010AE4F6
:100400000093360106E019E4EFE1F1E01083349641
:100410000A95E1F7EAEAFEE1E0933C01F0933D0141
:10042000E6E7FFE1E0934001F0934101E0ECFFE1FA
:10043000E0934401F0934501ECEFFFE1E0934801C4
:10044000F0934901E8E6F0E2E0935001F0935101A6
:10045000E4E7F1E2E0935801F0935901EEE2F2E2B1
:10046000E0936001F0936101EAE9F2E2E093680150
:10047000F0936901E2E4F3E2E0937001F09371011B
:10048000E2ECF3E2E0937801F0937901E0E9F4E241
:10049000E0938001F09381010CE308830EE30F8366
:1004A00008870FE0088BE6EFF2E0EEAFFFAF01EC5C
:1004B0000093640079DEF9DE31D10E941C0D0E94A8
:1004C000220C5ED566D5D9DE09DE04D60E87C0D5EE
:1004D000F5D50D8705E00A8BF98AF3D50B8F00233C
:1004E00011F00FEF098BF3D50F87F7D5098F0E9415
:1004F0000F0D00910302002331F40E94D70B0F3F30
:1005000011F40E94BF0AD7D50E8F002321F0F0927C
:100510000401F0920501D8D50C87002311F40FE0F7
:1005200001C007E00A870987A2D740D279807ED030
:10053000BAD709810715D9F30A950983C4D11DDEFD
:10054000789420D60E94CD0A1DD60E94370C6ED01A
:1005500095FF19C09F7DECE1F3E0EEAFFFAFECD467
:1005600000E5E7D3A0E4B1E0DAD363D061D30FA113
:100570000F3429F0BEDE0023C1F70FE4DAD3E6EF33
:10058000F2E0EEAFFFAF93FF26C00B85002319F515
:1005900001DE1BD50E94FA0C0C85002349F403E30D
:1005A000B2D3A0E3B1E09BD3ACE2B1E09CD305C0F1
:1005B00006E3A9D3A0E1B1E092D338D0BCD20EA11A
:1005C000023329F096DE0023C1F797D325D30E948A
:1005D000010DDEDDFCD490FDEDD5B9CFFF93EF9397
:1005E000EEADFFAD0995EF91FF9108950F921F9227
:1005F0000F931F932F933F934F936F938F93BF93BB
:10060000AF93FF93EF935F937F9310D07F915F91B0
:10061000EF91FF91AF91BF918F916F914F913F916A
:100620002F911F910F911F900F900895BAD024D051
:100630000895E0D021D008950F921F920F931F9339
:100640002F933F934F936F938F93BF93AF93FF93EA
:10065000EF935F937F93EDDF7F915F91EF91FF9138
:10066000AF91BF918F916F914F913F912F911F91BA
:100670000F911F900F90089592FF1EC01F81088553
:100680000F83011B19F00E3108F406C00D8D0023F5
:1006900011F419D101C057D11091040210FF05C007
:1006A00011FFA9D412FDAED406C0AEA5BFA50A2F76
:1006B0000B2B09F0A0D49B7F97FF08C08BD40D8D26
:1006C000002311F400D101C03ED19F7796FF02C0F4
:1006D00050DD9F7B94FF21C00A890A9511F492D4C2
:1006E00005E00A8B098D002311F001E043D69F7EBF
:1006F0000BA101FF12C0198D0D8510230B8D102346
:1007000049F00B81043031F4A4E1B1E0E0E5FDE112
:1007100000EFA0DC0BA10D7F0BA30895209A219A76
:10072000229A239A389A399A3A9A3B9A539A549A27
:10073000559A5D9A5C9A089538B1307F0895582F84
:10074000580D5B0D5B98052F5F70532B58B90295C0
:1007500005B9562F590D5C0D052F5F70532B02956F
:100760005C985C9A5B9A58B905B95C985C9A089554
:10077000562F580D5B0D5B98052F5F70532B58B9A2
:10078000029505B9582F590D5C0D052F5F70532B3D
:1007900002955C985C9A5B9A58B905B95C985C9A2A
:1007A00008951127A0E0B1E0A10FBF1DA10FBF1D4B
:1007B000A10FBF1DA10FBF1DED91FD91BD90CD906B
:1007C00013950985039510170CF013C00E2F0F2BEE
:1007D00049F385918823D1F3659145914423B1F381
:1007E0004F3F01F325912F934F932DD08F916F9110
:1007F000F4CF08951127ACE3B1E0A10FBF1DA10F05
:10080000BF1DA10FBF1DA10FBF1DED91FD91BD909B
:10081000CD90139514310CF014C00E2F0F2B59F3FB
:100820005D9A85918823C9F3659145914423A9F385
:100830004F3F09F325912F934F9305D08F916F91DF
:10084000F4CF5D9A089578DFDF01EFE9F3E0522FEE
:10085000561B08F45195042F081B08F40195051741
:1008600040F4E8EBF3E08627682786274227242711
:100870004227481730F484274827842762272627F1
:100880006227442E481A522E561A08F451942224F4
:1008900033246624621710F4639401C06A944817E5
:1008A00078F05D980995250C3F1C722D720D74151A
:1008B0003F041CF0660D24183F088395481790F7F5
:1008C000FD015D9A08950F921F921F930F932F932E
:1008D0003F93FF93EF9357D31981139519831C33DB
:1008E00041F00A8D002311F0FA8E23C069D0B1D0F7
:1008F00021C090611E85112321F4E0D50ED1B7D51A
:1009000018C0F9821A8113951A831C336CF01BA14D
:1009100012601BA3FA821B8113951B83FED01B81DF
:10092000183114F0FB8205C01C8D112311F4E3D59E
:100930009ED53DD0EF91FF913F912F910F911F9147
:100940001F900F9008951E85112339F11CD308853F
:100950000F8319811A9519831F3F41F00A8D0023D7
:1009600011F0FA8E19C02CD074D017C01BE3198374
:1009700090611A811A951A831F3F71F41BE31A8341
:100980001BA112601BA31B811A951B83C6D01B8160
:100990001F3F11F417E11B830AD008951C8D0D8DA4
:1009A000102B19F48BD503D00895089587D5B5D0B1
:1009B00003D03AD098D0089503D010D01DD0089518
:1009C000E8E4F5E2098115E0019FE00DF11D8F01DA
:1009D000E8E0F1E0008311839BD10895E4E7F6E2BB
:1009E0000A8119E0019FE00DF11D8F01ECE0F1E0BB
:1009F000008311838DD10895E0E9F8E20A811CE0BB
:100A0000E9D60F930B81E6D6022F25E0029F1F91B6
:100A1000100D29E0129FE00DF11D8F01E0E1F1E0E2
:100A20000083118375D1089514D029D03ED0089544
:100A3000000FE00FFF1D05911491000F111F089585
:100A4000ECE0FBE2F5DF08950F851EE300FD1AE4FC
:100A500008950981E2D6F4DFE0E2F1E0008311833A
:100A600057D1F2DF185B1283022FEADFECE1F1E0ED
:100A7000008311834DD1E8DF1C5A128308950A8147
:100A8000CCD6DEDFE8E2F1E00083118341D1DCDF88
:100A9000185D1283022FD4DFE4E2F1E000831183BA
:100AA00037D1D2DF1C5C128308950B810F8400FCC8
:100AB00005C0EAEFFBE2E00FFF1D0491AED6C0DFF8
:100AC000E0E3F1E00083118323D1BEDF195F1283DD
:100AD000022FB6DFECE2F1E00083118319D1B4DF1D
:100AE0001C5E128308950F85002369F4E8EDFAE295
:100AF0000B810C3014F0E0EFFAE2E0933801F09350
:100B000039010EE305C0F0923801F09239010AE490
:100B100000933A01009336010895E6ECFCE1E0937E
:100B20000102F09302020E8D002321F4E0930401F0
:100B3000F093050108950EA1033389F495FF03C0D6
:100B40009F7D8BD474C093FF72C004E3DCD0D5D0FA
:100B5000A8E2B1E0C4D0A4E2B1E0C5D068C00433DB
:100B600089F495FF03C09F7D6ED461C093FF5FC081
:100B700005E3C9D0C2D0A0E2B1E0B1D0ACE1B1E0B0
:100B8000B2D055C0053359F495FF03C09F7D51D4B1
:100B90004EC093FF4CC009E3B6D0AFD029C0063396
:100BA00069F495FF03C09F7D58D441C093FF3FC0B7
:100BB00007E3A9D0ACE0B1E092D039C0073369F4C3
:100BC00095FF03C09F7D3FD432C093FF30C008E340
:100BD0009AD0A8E0B1E083D02AC0083399F495FFF9
:100BE00003C09F7D26D423C093FF21C009E38BD08F
:100BF000A6EFBDE1A0931401B0931501A4E1B1E00B
:100C00006ED015C0093309F007C095FF03C09F7D62
:100C100072D404C093FF0BC051D4C9DE68D0A0E0E9
:100C2000B0E0A0931401B093150102E36CD00895D5
:100C3000E4E9FCE00FA10055102F110F110F000F78
:100C4000010FE00FFF1D95FF0AC09F7D05911591D3
:100C5000F80109950DAD03950DAF32DB1AC093FF76
:100C600018C0329605911591FF93EF93F8010DADE1
:100C7000002309F009950FA103950A350CF00FE444
:100C800058D0EF91FF91A591B5910A2F0B2B09F048
:100C900046D00895C201000044014E1868064C0178
:100CA000EE0602075401BC06D2065C010A071E07C5
:100CB0006401240738076C01400754077401A30638
:100CC000B5067C015C07740784017C07940700006B
:100CD0000895ED91FD9112970FEFBCD90895F9DFBA
:100CE000A8A7B9A70895F5DFAAA7BBA70895A8A547
:100CF000B9A5D6D9F8A6F9A60895AAA5BBA5D0D9B5
:100D0000FAA6FBA60895977F0EA3F1DFD9DA08951E
:100D1000A8A5B9A51FDAAAA5BBA51CDA0895D9DF35
:100D2000ACA7BDA70895ACA5BDA5BAD9FCA6FDA6E4
:100D30000895977F0FA3FDAEC3DAF5DF0895ACA544
:100D4000BDA508DA08950AAD019503950AAF01D053
:100D500008950AADE6E6FDE06BDEE4E7F1E000832E
:100D60001183EDDF0895BA11CF110AAD1E8D19F070
:100D700005D509E50FA308950EA9039507310CF0D9
:100D800004E10EAB01D008950EA90451EEE9FDE097
:100D90004FDEE4E5F1E000831183D1DF08956810B0
:100DA0008510A4100EA9109100020117B1F01631A0
:100DB00069F485D40EA91F85112321F0053159F05E
:100DC000A5D409C0043139F0A1D405C0063111F40D
:100DD00076D401C09BD409E50FA308950DA9019510
:100DE00003950DAB01D008950DA9002319F40CE370
:100DF00010E202C000E210E2ECE4F1E000831183B3
:100E00009EDF08950DA91B85011719F0E1D309E5AF
:100E10000FA308950FA9019503950FAB01D0089575
:100E20000FA9002319F402ED11E202C004E012E25E
:100E3000ECE5F1E00083118382DF08950E851FA9A0
:100E4000011709F01FD4089508AD0195039508AF67
:100E500001D0089508AD002319F00EE612E202C099
:100E600002E512E2E4E6F1E00083118368DF089511
:100E700008AD1D85011719F039D409E50FA30895B0
:100E800009AD0195039509AF01D0089509AD00237F
:100E900019F006E113E202C00AEF12E2ECE6F1E01B
:100EA000008311834CDF089509AD1B8D011719F0E4
:100EB00042D409E50FA308950E850E1108950BADD8
:100EC000019503950BAF01D008950BAD002319F0E8
:100ED00004E514E202C006E114E2ECE7F1E000836D
:100EE00011832DDF089508950BAD1C8D011719F0A6
:100EF000A0D309E50FA308950E850E1108950CAD3A
:100F0000019503950CAF01D008950CAD002319F0A5
:100F100002E015E202C004EC14E2E4E8F1E0008330
:100F200011830DDF089508950CAD1D8D011719F083
:100F300098D309E50FA308950B850DAB55DF0C85FC
:100F4000002311F016E105C014E10F85002309F01C
:100F500015E11EAB1093000217DF0E850FAB60DFAB
:100F60000D8508AF77DF0B8D09AF90DF0E8D0AAFCF
:100F7000F0DE0C8D0BAFA9DF0D8D0CAFC6DF089531
:100F8000569A5E9808950D8500FF4E9A08955E98D2
:100F9000089557985F9A089508A90F3F71F4E8AA39
:100FA000A9A9BAA90A2F0B2B41F4A8E1B1E0E0E905
:100FB000FDE100EF4FD8A9ABBAAB08950FEF08AB36
:100FC000A9A9BAA96DD8F9AAFAAAFF820895088535
:100FD0000F8308950C8D00FD0895AEA5BFA50A2FBF
:100FE0000B2B41F4A8E1B1E0EAEAFDE10FEF32D8C2
:100FF000AEA7BFA70895AEA5BFA552D8FEA6FFA66F
:1010000027D0089509890F3F71F0FF93EF93E2E134
:10101000FCE203950770098B000FE00FFF1D859020
:101020009490EF91FF910895ABA9BCA90A2F0B2BC7
:1010300041F4A0E0B1E0E6E3FBE100E50BD8ABABA7
:10104000BCAB0895ABA9BCA92BD8FBAAFCAA0895F8
:101050000BA106FD0EC00E85002329F4F0921801A5
:10106000F092190106C0E4E8FDE1E0931801F09365
:1010700019010895A7E0B0E016C0A0E0B0E013C0E9
:10108000A6E0B0E010C0A3E0B0E00DC0A2E0B0E088
:101090000AC0A4E0B0E007C0A1E0B0E004C0A5E051
:1010A000B0E001E000C000900402002019F400BD8F
:1010B00016E082D30895A7E0B0E012C0A0E0B0E04F
:1010C0000FC0A6E0B0E00CC0A3E0B0E009C0A4E00F
:1010D000B0E006C0A2E0B0E009C0A1E0B0E000C00E
:1010E00011E06AD30F3F09F40027089511E064D39B
:1010F0000F3F09F40E2D08950F9309818EE1080F1B
:101100000C330CF00C535AD4882329F467DA898104
:10111000081729F0F8CF10D48ED30F91089588E5E1
:101120000F9108958F934ED4882311F457DAFBCF93
:101130008F91F9D3089546D4882311F44FDAFBCF69
:1011400016D408958F933ED4882311F447DAFBCF49
:101150008F9118D0089536D4882311F43FDAFBCF4D
:1011600016D408950F932ED4882311F437DAFBCFC9
:101170000F91002319F0E6E0FEE2F9C3EAE0FEE297
:10118000F6C30895E2E0FEE2F2C3A5D895FF02C0DF
:101190009F7DF8D823DAADD80023C1F70895F5DF95
:1011A000F4DF0895C8DFCEDFF0DF0895C4DFCADFC3
:1011B000F6DF08958F931F930F932F933F93BF9361
:1011C000AF93FF93EF930F921F92B6D334D388352A
:1011D00009F08FC0E8E4FCE2AEDF8EDFA3DFB2DF10
:1011E000843509F43AC0843409F46BC0833509F4BA
:1011F00066C08C3411F47AD27CC0813411F442D2AE
:1012000078C0863511F4B0D274C0833411F4E0D1C3
:1012100070C08E3411F453D26CC0803511F476D284
:1012200068C0823411F487D264C0813511F401D2D0
:1012300060C0823511F415D25CC0863411F49ED2A0
:1012400058C0883411F4C2D254C08D3419F40E94AD
:10125000261B4FC0883579F1BDCFE2E7FCE26BDF9A
:1012600056D040F16ED159DC6DDFEAE8FCE263DF75
:101270004ED000F15ED166DFE2EAFCE25CDF47D0EF
:10128000C8F00E85002351F48F9389818F9389DAFA
:101290008F9109D109810817C9F38F9140D1EA8E46
:1012A00009810A9509830FDB9B7791DE4BDF0027CD
:1012B00061D004C07BDBE4ECFDE23DDF1AC06DD100
:1012C00018C0EAEBFCE237DF22D0A8F352D13ADFB4
:1012D000E2EDFCE230DF1BD070F343D133DFEAEE06
:1012E000FCE229DF14D038F334D12CDF002742D0C0
:1012F00000C028DFEA8E1F900F90AF91BF91EF9151
:10130000FF913F912F910F911F918F910895F4DEDE
:1013100009DF883511F4089408950DD0C0F3082F23
:10132000EBDE00DF8835B9F306D0D0F31AE0019F79
:10133000800D88940895803328F08A3318F4805300
:101340008894089508940895E2E2FCE2F4DE82E3D2
:10135000E9DE8EE2E7DE87E3E5DEF4DE089555D2CE
:101360008F9382958F705DD28D938F918F7059D2AC
:101370008D93089527D3882311F430D9FBCFFF93A1
:10138000EF93BF93AF930F93A5E0B2E011D080E24B
:101390008D9329D00F91002321F08DE08D938AE069
:1013A0008D93FD92F4D2AF91BF91EF91FF9108958B
:1013B0008C81D5DF8DE28D938D81EEE0FEE28A9502
:1013C000880F880FE80FFF1D85918D9385918D9370
:1013D00085918D938DE28D9382E38D9380E38D9340
:1013E0008E81BDDF08958B81BADF8AE38D938A8178
:1013F000B6DF8AE38D938981B2DF0895E3D2882333
:1014000011F4ECD8B7CFFF93EF93BF93AF930F9343
:10141000A5E0B2E0E8DF0F91002321F08DE08D938D
:101420008AE08D93FD92B3D2AF91BF91EF91FF917E
:101430000895098103950C3308F0002709830E9461
:101440006001B5DA08950A8103950C3308F000278E
:101450000A830E946001ABDA08950B81039508317D
:1014600008F000270B830E946001A1DA08950F9312
:101470008F9315E0E6D28F73B8D180320CF08E2DA9
:101480008C8317E0DED28F71B0D18D300CF08E2DB1
:101490008D8318E0D6D2A9D183360CF088278E83AD
:1014A0008F910F9108958F9312E0CBD28F779DD1BA
:1014B0008C330CF0882789838F9108958F9312E0E5
:1014C000C0D287FD69DD8F7790D18C330CF08827EF
:1014D000898313E0B6D28F7788D18C330CF08827BC
:1014E0008A8314E0AED28F7380D188310CF08827C4
:1014F0008B838F91089580910402882379F48981E8
:1015000084D112E0082FBFD28A817FD113E0082F47
:10151000BAD28B817AD114E0082FB5D208958F9377
:10152000082F0C3320F4898370D112E0ACD28F9154
:101530000895082F0C3320F48A8367D113E0A3D2D7
:101540000895082F083120F48B835FD114E09BD2DB
:101550000895082F003220F48C8357D115E093D2E0
:101560000895082F0C3020F48D834FD117E08BD2D3
:101570000895082F8E8349D118E085D208958827D1
:10158000CEDF8827D6DF8827DCDF81E0E2DF81E05D
:10159000E8DF8827EEDF83DD0895D6DE0027EADE68
:1015A00080E2C0DD82E50E85002309F081E4BADD2A
:1015B0000D85002311F48CE4B5DD0B8D002311F4AF
:1015C00082E4B0DD098D002311F086E5ABDD0895DE
:1015D0002F93E2E0FDE2AFDD0B85002339F01FD24F
:1015E000002722271A85E6E3FBE109C015D013D2B4
:1015F0000E2D2FEF8824992411E0EEE2F5E21987F1
:10160000E0930001F09301011B8D112309F4298B54
:101610000B87A8DD2F9108950C8D002321F01EE388
:1016200018871F83FC8E0D8D002309F0FD8EB6D91F
:1016300008950E8500FD04C0E2E8FDE27CDD10C0E7
:10164000E8E6FDE278DD0C8D002319F01EE30027AB
:1016500002C012E00E2D18871F830C8F83DD9ED9E8
:1016600008950E8500FD04C0E2E8FDE264DD09C0D6
:10167000E4E7FDE260DD0D8D019503950D8F72DDD0
:101680008DD90895E2E4FDE256DD0E85002339F0A0
:10169000C3DF0027F0921801F092190107C00395EB
:1016A000E4E8FDE1E0931801F09319010E87EEDC08
:1016B00059DD0091040200FF0E94C20108950B85CC
:1016C000002399F4E8E1FDE236DD0C85002319F0F2
:1016D00000271FE002C0039517E00C8719871A87BF
:1016E000D2DC019503953EDD18DA0895EAE2FDE2C9
:1016F00022DD0D85002311F0002702C0039547DC91
:101700000D87BBDC019503952DDD0895EAE3FDE22D
:1017100012DD0F85019503950F87BBDC1EE300FDED
:101720001AE4019503951EDD2F2D03D0DCD97CD959
:1017300008957AD90895E4E5FDE2FDDC0B8D01956D
:1017400003950B8F0F939CDC019503950BDD0F9197
:101750001B85112341F4002329F00FEF098B882406
:10176000992401C0F98A0895E0E3FDE2E4DC098DE3
:1017700001950395098F90DCF5DC0895E0EBFDE21F
:10178000DADC0E8D002331F00027E0910102F091A8
:10179000020203C00395E0E0F0E0E0930401F0935F
:1017A00005010E8F67DC01950395DCDC0895A5E04B
:1017B000B0E011E001D00895A1BDB2BD119611FDB8
:1017C000FA9A1FBBF999FECF00B50895EEE3FEE249
:1017D000B2DC0895222738E0000F221F211710F0F5
:1017E0000395211B3A95C1F708950F921F920F930D
:1017F0008F9382958F700AE0809F002D8F918F705C
:10180000800F0F911F900F900895082F1AE0E2DFCC
:1018100007700295022B802F08951AE0DBDF077016
:101820000895FF93EF93EAEEFBE2E80FFF1D84912A
:10183000EF91FF910895813624F08B3710F400E288
:10184000801B089510E41093C400F092C500F0923C
:10185000C00018E41093C10016E01093C200EB8A98
:10186000FF8AF88EFC8AFD8A1FEF1E8B0895109167
:10187000C10010691093C10008950F930FB70F9323
:101880001F93FF93EF930E890F3F79F00395E5E0E7
:10189000F2E0E00FFF1D1081112319F40FEFEB8A26
:1018A00002C01093C6000E8B12C0EC89FD890E2F6A
:1018B0000F2B39F0EF5FFF4F1491112321F4FC8AB5
:1018C000FD8AEB8A04C01093C600EC8BFD8BEF9170
:1018D000FF911F910F910FBF0F9118950F930FB7A5
:1018E0000F930BA102FD0C94851B1F932F933F9325
:1018F000FF93EF932091C6000F89302F03950F704F
:10190000188D011739F00F8BE5E8F2E0E30FFF1DAA
:1019100020839160EF91FF913F912F911F910F9143
:101920000FBF0F9118950F930B890023E9F3FB8AE2
:101930008093C6000F91089590FFFECF0F931F93E1
:10194000FF93EF931F89088D8827011751F0E5E871
:10195000F2E0E00FFF1D808103950F70088F0117E3
:1019600009F49E7FEF91FF911F910F9108950F93BE
:10197000FF93EF930B890023E9F3FB8AEC8BFD8B3C
:1019800004910093C600EF91FF910F9108950F937A
:10199000FF93EF930B890023E9F3FB8AFE8AE5E0CE
:1019A000F2E00081002321F40FEF0E8BEB8A02C0DE
:1019B0000093C600EF91FF910F910895882790FD45
:1019C000839508958B8908951F930F9328D01FE066
:1019D00000E459D01EE001E856D011E001E153D0F7
:1019E0000F911F9108951FE000E44DD011E001E137
:1019F0004AD008951EE000E846D011E000E143D04F
:101A000008951FE000E43FD01EE001E83CD011E063
:101A100001E139D008951DE000E835D008951DE0BA
:101A2000002731D0089500000000000000000000F1
:101A300000000000000008953C9A3D9A449A459A9F
:101A400008953F9333273A9519F4E092030217C0A3
:101A5000B1F067D0E8DF02EA3FD0E5DF33D098F39A
:101A6000012F3AD0E0DF2ED070F355D05AD003EAE0
:101A700033D0D9DF27D038F33CD0449A459A4BD0A5
:101A8000802F3F9108953F9333273A9519F4E092C0
:101A9000030215C046D0C7DF0F9302EA1DD0C3DF93
:101AA00011D00F9190F30F93012F16D00BD00F91FF
:101AB00060F30F9311D006D00F9138F300002BD0B4
:101AC0003F9108953C98449A0894459AACDF349B22
:101AD000889445983C9A08953F9338E0449A000FC3
:101AE00008F04498459A9FDF45983A95B9F73F9199
:101AF00008953F933C98449A00E038E0459A089452
:101B000092DF349B8894001F45988DDF3A95B1F79A
:101B10003C9A3F9108954498459A00000000449AE9
:101B20000895449A459A000000004498000000007F
:101B30004598000008957AEB7AD90080E883EB8914
:101B4000EB8CE88CE580D98CD900862483277D270F
:101B50007A247A187D1583158618861B831E7D1EB0
:101B60007A1B00E086E389E989EC86EC83E980EC66
:101B70007DEC7AE977E377E07A00E380E980001F83
:101B8000831C801C8016801383138616891C891F72
:101B9000861F7A1C771677137A0080FE80F2008DFC
:101BA000FE8CF9009AFC99F700A6F8A5F400B3F4AE
:101BB000B1EF00BFEEBAE500CAE6C7E200D4DED05E
:101BC000DA00DDD5D9D100E5CBE1C800EDBFE4BA3C
:101BD00000F3B4EEB200F7A7F3A600FB9BF69A0061
:101BE000FD8EF88D00FD80F18000FD73F87400FB20
:101BF00066F66700F75AF35B00F34DEE4F00ED41D8
:101C0000E44600E536E13900DD2CD93000D423D09C
:101C10002700CA1BC71F00BF13BA1C00B30DB112A7
:101C200000A609A50D009A05990A008D038C0800ED
:101C30007F037F0F0072037308006505660A005971
:101C4000095A0D004C0D4E12004113461C00351B65
:101C5000381F002B232F2700222C2630001A361E77
:101C6000390012421B47000C4D114F00085A0C5B03
:101C7000000466096700027307740002810E810088
:101C8000028E078D00049B099A0008A70CA6000C81
:101C9000B411B20012BF1BBA001ACB1EC80022D565
:101CA00026D1002BDE2FDA0035E638E20040EE4583
:101CB000E5004CF44EEF0059F85AF40065FC66F765
:101CC0000072FE73F9FFB5E4B5D20000D2BBD5BEF9
:101CD000DBBEDEBBDEB8D2ACDEAC0000E04CD44CE8
:101CE000DD55DD430000B831AC31AC28B528B8254E
:101CF000B822B51FAF1FAC22000047315331532E1D
:101D0000502B4D254D1F0000224C1F4F1F522255B6
:101D100028552B522B4F284C224C1F491F4622433B
:101D200028432B462B49284C000021BE21AC000043
:101D300027BB2ABE30BE33BB33AF30AC2AAC27AF93
:101D400027BB000049E449D2000053E453D2FF000E
:101D5000B2A4B2A6BAA6BA9AB29AB29C00BE9ABE71
:101D60009EC49EC49ABE9A00C49AC4A600C79AC7CD
:101D7000A6CDA6CFA4CFA2CDA0C7A000CDA0CF9EB8
:101D8000CF9AFF007CBA80C684BA0082BE7EBEFFB6
:101D90007CBA7CC682C684C484C282C07CC082C035
:101DA00084BE84BC82BA7CBAFF007CBA7CC682C680
:101DB00084C484C282C07CC0FF00A999AC99AD984C
:101DC000AD94AC93A993A99900B999B599B593B974
:101DD0009300B896B59600C093C099C297C499C4B1
:101DE0009300CB98CC99CE99CF98CF94CE93CC93A7
:101DF000CB94CB98FF003A933A993D993E983E9701
:101E00003D963A960046994694479349934A9400E2
:101E10004A994A9300569855995399529852975314
:101E200096559656955694559353935294005E99B1
:101E30005E93005E96629600629362990076997A4C
:101E400099007899789300829883998599869886E5
:101E5000948593839382948298009E989D999B99F0
:101E60009A989A979B969D969E959E949D939B93E8
:101E70009A9400A699AA9900A899A89300B293B43D
:101E800099B69300B595B39500BE93BE99C199C21A
:101E900098C297C196BE9600C196C295C29300CAD9
:101EA00099CE9900CC99CC93FF0029EC2FEC31EA24
:101EB00031E22FE029E029EC0035EC35E237E03B58
:101EC000E03DE2003DEC3DE00041EC49EC0045EC3A
:101ED00045E00055EA53EC4FEC4DEA4DE24FE0533C
:101EE000E055E20059EC59E00059E661E60061E096
:101EF00061EC0065EC6DEC0069EC69E00071E0718B
:101F0000EC77EC79EA79E877E671E60077E679E450
:101F100079E0007DEA7FEC83EC85EA85E283E07F6F
:101F2000E07DE27DEA0089E089EC91E091EC0097A8
:101F3000E09BE00099E099EC0097EC9BEC00A1ECB1
:101F4000A9E000A9ECA1E000B9ECBDE0C1EC00C53E
:101F5000EAC7ECCBECCDEACDE8C5E0CDE000D3E0BC
:101F6000D3E4D7E4D7E0D3E000DDECE5ECE5EAE349
:101F7000E8E1E4E1E0FF29C229CE2FCE31CC31CA1D
:101F80002FC829C82FC831C631C42FC229C2003575
:101F9000CC37CE3BCE3DCC3DC43BC237C235C43539
:101FA000CC0041CC43CE47CE49CC49C447C243C202
:101FB00041C441CC004DCE55CE0051CE51C2FF00A0
:101FC00029BA2FBA31B831B02FAE29AE29BA003DA7
:101FD000BA35BA35AE3DAE003BB435B40041AE4182
:101FE000BA45B649BA49AE004DB84FBA53BA55B81A
:101FF00055B053AE4FAE4DB04DB8FF0031A42FA633
:102000002BA629A4299C2B9A2F9A319C00359A390A
:10201000A63D9A003B9E379E0041A6419A499AFFF1
:1020200059A45BA65FA661A4619C5F9A5B9A599CC8
:1020300059A400659A65A66D9A6DA6FF59A45BA682
:102040005FA661A4619C5F9A5B9A599C59A4006D3C
:10205000A665A6659A0065A06BA00079A671A67119
:102060009A0071A077A0FF002986299231863192CB
:10207000003592358837863B863D88003D923D8607
:102080000041864192458E499249860055924D9273
:102090004D86558600538C4D8C00598659925F921F
:1020A0006190618E5F8C598C005F8C618A618600C3
:1020B00067866B8600698669920067926B920079E9
:1020C000907792739271907188738677867988FF82
:1020D0008D928D8600959097929B929D909D8E9566
:1020E000869D8600A192A18600A18CA98C00A9865C
:1020F000A99200AD86AD92B392B590B58EB38CAD7A
:102100008C00B38CB58AB586FF0089908B928F9234
:102110009190918E89869186009D8C958C9B929B47
:102120008600A192A18600A18CA98C00A986A99203
:1021300000AD86AD92B392B590B58EB38CAD8C00E8
:10214000B38CB58AB586FF0089908B928F9291905F
:1021500091888F868B8689888990009D929592952B
:102160008600958C9B8C00A992A192A18600A18CDF
:10217000A78CFF002972297E2D7A317E31720035BD
:1021800072397E3D72003B76377600497C477E434C
:102190007E417C417A437847784976497447724357
:1021A000724174004D7E557E00517E517200617EF9
:1021B000597E59726172005F785978006572657E48
:1021C0006B7E6D7C6D7A6B786578006B786D766D63
:1021D00072FF7D727D7E837E857C857A83787D78B3
:1021E0000083788576857200897E917E008D7E8D54
:1021F00072009D7C9B7E977E957C957497729B72F6
:102200009D74FF007D72817E85720083767F7600EB
:10221000897E8D72917E009572957E9B7E9D7C9DC0
:102220007A9B789578009B789D769D72FF00296A4D
:10223000295E315E003D6A356A355E3D5E003B6475
:10224000356400416A476A49684960475E415E41BA
:102250006AFF59685B6A5F6A616861605F5E5B5EC6
:102260005960596800655E656A6D5E6D6AFF596800
:102270005B6A5F6A616861605F5E5B5E5960596856
:10228000006D6A656A655E0065646B6400796A71F9
:102290006A715E0071647764FF00294A29562F56DF
:1022A000315431522F5029502F50314E314C2F4A3A
:1022B000294A003556354C374A3B4A3D4C003D567D
:1022C0003D4A00414A4156475649544952475041B8
:1022D00050004750494E494A004D4A4D56554A55BF
:1022E00056005B4A5F4A005D4A5D56005B565F568A
:1022F00000654A65566D4A6D56FF7D547F5683567C
:102300008554854C834A7F4A7D4C7D5400894A8997
:1023100056914A9156FF7D547F5683568554854C7D
:10232000834A7F4A7D4C7D540091568956894A00E4
:1023300089508F50009D569556954A0095509B5058
:10234000FF0029422F42314031382F3629362942A9
:102350000037363B3600393639420037423B4200BF
:1023600041364542493600473A433A004D424D36E0
:102370005536FF006D426542653600653C6B3C009A
:102380007142713873367736793800794279360080
:102390007D427D36853600894289369136FF653625
:1023A0006542693E6D426D3600733677360075368C
:1023B00075420073427742007D367D428536854204
:1023C000FF00312C2F2E2B2E292C292A2B282F28A9
:1023D000312631242F222B222924003522352E3B71
:1023E0002E3D2C3D2A3B28352800492E412E4122E6
:1023F0004922004728412800552E4D2E4D225522B6
:102400000053284D2800592E5F2E612C61245F2235
:102410005922592EFF007122712E7922792E007DCA
:102420002C7F2E832E852C852483227F227D247D64
:102430002C008922892E8F2E912C912A8F28892871
:10244000008F2891269122009522952E992A9D2E63
:102450009D22FF00792E712E7122007128772800AD
:102460007D22812E85220083267F2600912C8F2EAF
:102470008B2E892C892A8B288F28912691248F22B4
:102480008B22892400952E9D2E00992E9922FF00E3
:10249000291A2F1A311831102F0E290E291A003738
:1024A0000E3B0E00390E391A00371A3B1A00410E46
:1024B000411A471A4918491647144114004714494C
:1024C00012490EFF590E591A610E611A00651867FC
:1024D0001A6B1A6D186D106B0E670E65106518007B
:1024E000710E711A771A79187916771471140077AA
:1024F000147912790E007D0E7D1A8116851A850ECB
:10250000FF00590E591A5F1A611861165F145914A9
:10251000005F146112610E006D1A651A650E6D0E72
:10252000006B14651400711A750E791AFF0001FE14
:102530000101FE01FEFE01FEFE010101FEFE01FEA3
:102540000101FE01FEFEFF0080EC8080FF8BEC802D
:1025500080FF96EA8080FFA1E78080FFABE3808068
:10256000FFB6DE8080FFBFD88080FFC8D18080FFAB
:10257000D0C98080FFD7C08080FFDDB68080FFE2B9
:10258000AC8080FFE6A28080FFE9978080FFEB8C23
:102590008080FFEB808080FFEB758080FFE96A80A0
:1025A00080FFE65F8080FFE2558080FFDD4A80800B
:1025B000FFD7418080FFD0388080FFC8308080FF07
:1025C000BF298080FFB6238080FFAB1E8080FFA1E3
:1025D0001A8080FF96178080FF8B158080FF801502
:1025E0008080FF74158080FF69178080FF5E1A80ED
:1025F00080FF541E8080FF4A238080FF4029808016
:10260000FF37308080FF2F388080FF28418080FF97
:10261000224B8080FF1D558080FF195F8080FF1650
:102620006A8080FF14758080FF14808080FF148C86
:102630008080FF16978080FF19A28080FF1DAC80EC
:1026400080FF22B68080FF28C08080FF2FC9808055
:10265000FF37D18080FF40D88080FF49DE8080FF37
:1026600054E38080FF5EE78080FF69EA8080FF742A
:10267000EC8080FF828080E67E808280FF81808A7D
:10268000E67E818180FF818095E47E818180FF816B
:10269000809FE27E818180FF8180A9DE7E818180B2
:1026A000FF817FB3D97E82817FFF817FBBD37E8212
:1026B000817FFF817FC4CC7E82817FFF817FCBC5FC
:1026C0007E82817FFF817FD2BC7E82817FFF807F7F
:1026D000D8B37F82807FFF807FDDAA7F82807FFFEB
:1026E000807FE1A07F82807FFF807FE3967F828072
:1026F0007FFF807FE58B7F82807FFF7F7EE580800C
:10270000827F7EFF7F7FE57680827F7FFF7F7FE312
:102710006B80827F7FFF7F7FE16180827F7FFF7F91
:102720007FDD5780827F7FFF7E7FD84D81827E7FD5
:10273000FF7E7FD24581827E7FFF7E7FCB3C818280
:102740007E7FFF7E7FC43581827E7FFF7E7FBB2EB2
:1027500081827E7FFF7E7FB32881827E7FFF7E80A5
:10276000A92381817E80FF7E809F1F81817E80FFE3
:102770007E80951D81817E80FF7E808A1B81817E87
:1027800080FF7E817F1B82807E81FF7E81751B8121
:10279000807E81FF7E816A1D81807E81FF7E8160D7
:1027A0001F81807E81FF7E81562381807E81FF7E16
:1027B000814D2881807E81FF7E82442E817F7E82B2
:1027C000FF7E823B35817F7E82FF7E82343C817F2B
:1027D0007E82FF7E822D45817F7E82FF7F82274E13
:1027E000807F7F82FF7F822257807F7F82FF7F8270
:1027F0001E61807F7F82FF7F821C6B807F7F82FFD4
:102800007F821A76807F7F82FF80821A817F7E801E
:1028100082FF80821A8B7F7F8082FF80821C967F5E
:102820007F8082FF80821EA07F7F8082FF80822245
:10283000AA7F7F8082FF808227B37F7F8082FF8193
:10284000822DBC7E7F8182FF818234C57E7F818222
:10285000FF81823BCC7E7F8182FF818244D37E7F59
:102860008182FF81824CD97E7F8182FF818156DE09
:102870007E808181FF818160E27E808181FF818114
:102880006AE47E808181FF818175E67E808181FF9F
:10289000828080BC7E808280FF818086BC7E818138
:1028A00080FF81808CBB7E818180FF818092BA7E97
:1028B000818180FF818098B77E818180FF817F9EAA
:1028C000B47E82817FFF817FA3B17E82817FFF8181
:1028D0007FA8AD7E82817FFF817FACA97E82817FD0
:1028E000FF817FB0A47E82817FFF807FB39E7F8245
:1028F000807FFF807FB6997F82807FFF807FB99342
:102900007F82807FFF807FBA8D7F82807FFF807F84
:10291000BB877F82807FFF7F7EBB8080827F7EFF40
:102920007F7FBB7A80827F7FFF7F7FBA7480827FC8
:102930007FFF7F7FB96E80827F7FFF7F7FB6688059
:10294000827F7FFF7E7FB36281827E7FFF7E7FB04A
:102950005D81827E7FFF7E7FAC5881827E7FFF7E9D
:102960007FA85481827E7FFF7E7FA35081827E7FFD
:10297000FF7E7F9E4D81827E7FFF7E80984A81818F
:102980007E80FF7E80924781817E80FF7E808C46A4
:1029900081817E80FF7E80864581817E80FF7E8171
:1029A0007F4582807E81FF7E81794581807E81FFA7
:1029B0007E81734681807E81FF7E816D4781807E2E
:1029C00081FF7E81674A81807E81FF7E81624D81A9
:1029D000807E81FF7E825C50817F7E82FF7E825777
:1029E00054817F7E82FF7E825358817F7E82FF7E6C
:1029F000824F5D817F7E82FF7F824C63807F7F82FA
:102A0000FF7F824968807F7F82FF7F82466E807F62
:102A10007F82FF7F824574807F7F82FF7F82447A3E
:102A2000807F7F82FF808244817F7E8082FF8082E0
:102A300044877F7F8082FF8082458D7F7F8082FFF9
:102A4000808246937F7F8082FF808249997F7F804A
:102A500082FF80824C9E7F7F8082FF81824FA47E96
:102A60007F8182FF818253A97E7F8182FF8182578D
:102A7000AD7E7F8182FF81825CB17E7F8182FF811A
:102A80008261B47E7F8182FF818167B77E80818190
:102A9000FF81816DBA7E808181FF818173BB7E80E1
:102AA0008181FF818179BC7E808181FF24532455FF
:102AB00026552653245300244F244D264D264F24BB
:102AC0004F004453445546554653445300444F44E5
:102AD0004D464D464F444FFF644B68576C4B006A60
:102AE0004F664F00704B705774537857784BFF0008
:102AF000644B64576A576C556C536A5164510000BB
:102B0000704B705774537857784BFF0090159A1597
:102B10009D15A515B315B815C215CF15D615E71512
:102B2000040C060E0A0E0C0C0C040A020602040425
:102B3000040CFF00080E0802FF00040C060E0A0E2B
:102B40000C0C0C0A04020C02FF00040C060E0A0E08
:102B50000C0C0C0A0A080C060C040A0206020404F7
:102B60000006080A08FF0C0804080A0E0A02FF0003
:102B70000C0E040E04080A080C060C040A020602D5
:102B80000404FF000C0C0A0E060E040C04040602DA
:102B90000A020C040C060A0806080406FF00040ECC
:102BA0000C0E0C0C0A0A08060802FF000608040AAC
:102BB000040C060E0A0E0C0C0C0A0A080608040681
:102BC000040406020A020C040C060A08FF000C0AA0
:102BD0000A080A080608040A040C060E0A0E0C0C61
:102BE0000C040A0206020404FF003031323334358B
:102BF000363738394142434445460C010203040547
:102C0000060708090A0B0C01020304050607080958
:102C10000A0B0000010001010001FF01FF00FFFF9E
:102C200000FF447574636874726F6E697820415652
:102C300052204F7363696C6C6F73636F70652043D0
:102C40006C6F636B20560000456E74657220636F75
:102C50006D6D616E642028412C422C432C442C461F
:102C60002C482C4C2C4E2C502C532C542C56293A9E
:102C70000000456E746572203220646967697420B3
:102C8000686F7572733A20202000456E746572205B
:102C900032206469676974206D696E757465733A72
:102CA0002000456E74657220322064696769742063
:102CB0007365636F6E64733A2000456E74657220AD
:102CC0003220646967697420796561723A20202036
:102CD0002000456E74657220322064696769742033
:102CE0006D6F6E74683A20202000456E7465722006
:102CF00032206469676974206461793A2020202059
:102D0000200043616C6962726174696F6E2050616A
:102D1000747465726E2000004E756D657269632073
:102D2000646973706C61792000004C454420000098
:102D3000566572626F7365200000414D2F504D2023
:102D4000000041565220436C6F636B204D617374D9
:102D5000657220004275726E2D696E205072657624
:102D6000656E74696F6E200046617374204D6F64E8
:102D70006520000052657665727365204D6F64654D
:102D80002000526571756573746564206D6F6465AC
:102D90002072657175697265732041565220636CAB
:102DA0006F636B204D6173746572204D6F646500B5
:102DB000416C6C2044696769747320646973706C3A
:102DC0006179200043616E63656C206F72205469E5
:102DD0006D656F7574004E6F7420456E7465726911
:102DE0006E672044656D6F204D6F64650000505024
:102DF00053207369676E616C2069676E6F726564DA
:102E000000000D0A00004F6E00004F6666004A6128
:102E10006E1F4665621C4D61721F4170721E4D61CE
:102E2000791F4A756E1E4A756C1F4175671F536581
:102E3000701E4F63741F4E6F761E4465631F44758A
:102E400074636874726F6E6978204F7363696C6C19
:102E50006F73636F706520436C6F636B2048656CA4
:102E6000703A0D0A413A20546F67676C65204D61D6
:102E70007374657220436C6F636B20626574776551
:102E8000656E2041565220616E64205254430D0AF3
:102E9000423A20546F67676C65204275726E2D69E7
:102EA0006E2070726576656E74696F6E0D0A433AB6
:102EB00020446973706C61792043616C696272614E
:102EC00074696F6E207061747465726E0D0A443A95
:102ED000204368616E676520446174650D0A463A57
:102EE00020546F67676C6520416C6C20446967698A
:102EF000747320446973706C61790D0A4C3A2054E4
:102F00006F67676C65204C454420626C696E6B6925
:102F10006E670D0A4E3A20546F67676C65204E75D8
:102F20006D6572696320446973706C6179200D0A64
:102F3000503A20546F67676C6520414D2F504D20EB
:102F40000D0A533A20446973706C6179205374619F
:102F5000747573200D0A543A204368616E676520CA
:102F600054696D650D0A563A20546F67676C652089
:102F7000566572626F7365204F75747075740D0AB3
:102F80000000EAEBFDE1E0931401F09315010895D0
:102F9000E0E0F0E0E0931401F093150108950C8552
:102FA0000023D9F50E945F0B36C00C850023A9F1E0
:102FB0000E945F0B30C00F85002379F50E94860BBD
:102FC0002AC00F85002349F10E94860B24C00E8D74
:102FD000002319F50E94BE0B1EC00E8D0023E9F0E0
:102FE0000E94BE0B18C00D850023B9F40E94760B19
:102FF00012C00D85002389F00E94760B0CC00B8552
:10300000002361F00E94E80A06C00B85002331F41A
:103010000E94E80A00C00E94A20800C00895098D1D
:103020000023E1F30E94B40BF6CF098D0023B1F722
:103030000E94B40BF0CF0E85002381F30E94420B57
:10304000EACF0E85002351F70E94420BE4CF0C8D8E
:10305000002321F30E94190BDECF0C8D0023F1F623
:103060000E94190BD8CF0D8D0023C1F20E94310BA5
:10307000D2CF0D8D002391F60E94310BCCCF089555
:10308000F98A08950E94FB0708950E94EA070895AF
:103090000E94DE0708950E94CC07089501E0009386
:1030A00004020E94C117D3DFDEDFA9DFE6EFF2E002
:1030B000EEAFFFAFE6E5F2E30E94D208EAEFF2E3FB
:1030C0000E94D2080E94CF170E94E717E8E2F3E3BC
:1030D0000E94D2080E94ED17EAE4F3E30E94D208AE
:1030E0000E94DB170E94D517E8E6F3E30E94D2089E
:1030F0000E94E117EAE8F3E30E94D208ECEAF3E366
:103100000E94D2080E94DB170E94C5080E94E717A0
:103110000E94C5080E94E1170E94C5080E94ED1791
:103120000E94CF170E94C5080E94ED170E94D51774
:103130000E94C5080E94E7170E94CF170E94C50889
:103140000E94ED170E94E1170E94D5170E94C50842
:103150000E94F317E8ECF3E30E94D6080E94F917E7
:10316000E2EEF3E30E94D6080E940518E6EFF3E3CF
:103170000E94D6080E94FF17E0E1F4E30E94D608FF
:103180000E942118E2E2F4E30E94D6080E942D1862
:10319000E4E5F4E30E94D6080E94CF080E942718B5
:1031A000E6E6F4E30E94D6080E943918EAE7F4E361
:1031B0000E94D6080E942D18ECE8F4E30E94D6087D
:1031C0000E94CF080E940C0B009304020E944B182F
:1031D000EAECF4E30E94D6080E94CF0803E00093D3
:1031E00004020E9448180E944518ECE1F5E30E9491
:1031F000D6080E94CF080E9442180E941408ECE6EC
:10320000F5E30E94D60805E0009304020E9422081C
:103210000E944018EAE8F5E30E94D6080E94CF0811
:10322000F09204020E943F18ECE1F3E0EEAFFFAF32
:10323000E6EDF2E30E94D6080E94CF08E6EFF2E046
:10324000EEAFFFAFEAEEF5E30E94D2080E94C81786
:103250000E94C2010895546869732064656D6F20EF
:103260006D6F64652073686F777320736F6D652071
:103270006F6620746865206361706162696C69744F
:10328000696573206F66207468652044757463688F
:1032900074726F6E69780D0A415652204F736369DC
:1032A0006C6C6F73636F706520436C6F636B2E2063
:1032B00049742070726573657276657320746865F1
:1032C000207374617465206F6620796F7572206356
:1032D0006C6F636B2E004865726520796F75206393
:1032E000616E2073656520746865206F6E2D736351
:1032F0007265656E206D656E75004865726520614A
:10330000726520736F6D65206F6620746865204359
:103310006C6F636B20446973706C61797320737593
:1033200070706F7274656400416E616C6F672043EA
:103330006C6F636B2077697468206D696E696D616D
:103340006C206469676974730000416E616C6F671B
:1033500020436C6F636B207769746820616C6C200C
:10336000646967697473000041646420746865204F
:10337000323420686F757273206E756D6572696383
:1033800020646973706C617900004F72206164641D
:103390002074686520414D2F504D206E756D65720B
:1033A000696320646973706C617900004D697820ED
:1033B000616E64204D6174636820617320796F755C
:1033C00020706C65617365005475726E2074686559
:1033D000204C454420626C696E6B696E67206F6695
:1033E0006600416E64207475726E2069742062619B
:1033F000636B206F6E005475726E206F6E20436198
:103400006C6962726174696F6E204D6F6465000053
:103410005475726E206974206261636B206F6666FA
:10342000000054686520274127206F6E207468656E
:103430002073636F7065206D65616E732041565215
:1034400020436C6F636B204D6173746572204D6F08
:10345000646500004D616B652054696D6520676F80
:103460002066617374004D616B652054696D652041
:10347000676F206E6F726D616C004D616B652054DB
:10348000696D6520676F206261636B004D616B65DC
:103490002054696D6520676F206261636B206661EF
:1034A00073742100566572626F7365206F75747056
:1034B0007574206973206F6E65206F6620796F7553
:1034C00072206F7074696F6E730054686520626C4F
:1034D000696E6B696E67204220776F756C64206936
:1034E0006E6469636174652061206C6F772052544B
:1034F00043206261636B75702062617474657279D8
:103500002C20627574206E6F772069742773206A8F
:1035100075737420612064656D6F00005468697371
:1035200020626C696E6B696E67205020696E6469F9
:1035300063617465732074686174207468652031F8
:1035400020505053207369676E616C206973206D41
:10355000697373696E672E20416761696E2C206AFA
:1035600075737420612064656D6F000057696C6C21
:1035700020746869732067657420796F75722061A3
:103580007474656E74696F6E3F004275726E206967
:103590006E2070726576656E74696F6E206D6F76E1
:1035A00065732074686520646973706C617920614B
:1035B0002074696E79206269742C206E6F726D615F
:1035C0006C6C792065766572792035206D696E7531
:1035D0007465732062757420686572652065766510
:1035E0007279207365636F6E6400576520686F7031
:1035F0006520796F7520656E6A6F796564207468DF
:1036000069732064656D6F2E205468616E6B20793C
:103610006F7520666F72207573696E6720746869B4
:103620007320447574636874726F6E697820436C9C
:103630006F636B001BA114601BA3F8940E94CA0067
:103640000E94F2000E94860178940895F3DFE0E082
:10365000F8E350E040E06DEF73E280E05B985C9847
:10366000460F571FE81F1491012F1F7018B90295BC
:1036700005B9F6CF0F930091C00005FFFCCF0F9165
:103680000093C60008958F930F9302950F70802FBB
:103690000E94110C082FEEDF0F910F70802F0E94F7
:1036A000110C082FE7DF8F91089506E40E943A1B62
:1036B00000270E94431B082F0E94431B072F0E94D4
:1036C000431B062F0E94431B0DE00E943A1B0AE099
:1036D0000E943A1B08956F5F7F1D8F1D08956C59DE
:1036E0007F1D8F1D089504E6FADF0A95E9F7089516
:1036F00061507F098F09089564567F098F090895E5
:1037000004E6FADF0A95E9F708950091C6000E94E1
:103710003A1B0B3211F4DFDF32C0053711F4DFDF63
:103720002EC0053511F4DFDF2AC00D3211F4E0DFC1
:1037300026C0043611F4E0DF22C0043411F4E0DFC7
:103740001EC00F3309F41BC0013319F4E0E0F8E3A5
:1037500016C0023319F4E0E0F9E311C0033319F4A1
:10376000E0E0FAE30CC0043319F4E0E0FBE307C047
:10377000013729F40BA10B7F0BA30E94C20195DF37
:083780000F910FBF0F91189586
:10380000808386898C8F9295989C9FA2A5A8ABAE49
:10381000B0B3B6B9BCBFC1C4C7C9CCCED1D3D5D85B
:10382000DADCDEE0E2E4E6E8EAECEDEFF0F2F3F514
:10383000F6F7F8F9FAFBFCFCFDFEFEFFFFFFFFFFC9
:10384000FFFFFFFFFFFFFEFEFDFCFCFBFAF9F8F7B0
:10385000F6F5F3F2F0EFEDECEAE8E6E4E2E0DEDCC8
:10386000DAD8D5D3D1CECCC9C7C4C1BFBCB9B6B3E1
:10387000B0AEABA8A5A29F9C9895928F8C898683A9
:10388000807C797673706D6A6763605D5A575451B6
:103890004F4C494643403E3B383633312E2C2A2785
:1038A0002523211F1D1B1917151312100F0D0C0AAC
:1038B00009080706050403030201010000000000D7
:1038C00000000000000001010203030405060708D0
:1038D000090A0C0D0F1012131517191B1D1F212398
:1038E00025272A2C2E313336383B3E404346494C5F
:1038F0004F5154575A5D6063676A6D707376797C77
:10390000000102030405060708090A0B0C0D0E0F3F
:10391000101112131415161718191A1B1C1D1E1F2F
:10392000202122232425262728292A2B2C2D2E2F1F
:10393000303132333435363738393A3B3C3D3E3F0F
:10394000404142434445464748494A4B4C4D4E4FFF
:10395000505152535455565758595A5B5C5D5E5FEF
:10396000606162636465666768696A6B6C6D6E6FDF
:10397000707172737475767778797A7B7C7D7E7FCF
:10398000808182838485868788898A8B8C8D8E8FBF
:10399000909192939495969798999A9B9C9D9E9FAF
:1039A000A0A1A2A3A4A5A6A7A8A9AAABACADAEAF9F
:1039B000B0B1B2B3B4B5B6B7B8B9BABBBCBDBEBF8F
:1039C000C0C1C2C3C4C5C6C7C8C9CACBCCCDCECF7F
:1039D000D0D1D2D3D4D5D6D7D8D9DADBDCDDDEDF6F
:1039E000E0E1E2E3E4E5E6E7E8E9EAEBECEDEEEF5F
:1039F000F0F1F2F3F4F5F6F7F8F9FAFBFCFDFEFF4F
:103A000000020406080A0C0E10121416181A1C1EC6
:103A100020222426282A2C2E30323436383A3C3EB6
:103A200040424446484A4C4E50525456585A5C5EA6
:103A300060626466686A6C6E70727476787A7C7E96
:103A400080828486888A8C8E90929496989A9C9E86
:103A5000A0A2A4A6A8AAACAEB0B2B4B6B8BABCBE76
:103A6000C0C2C4C6C8CACCCED0D2D4D6D8DADCDE66
:103A7000E0E2E4E6E8EAECEEF0F2F4F6F8FAFCFE56
:103A8000FFFDFBF9F7F5F3F1EFEFEBE9E7E5E3E134
:103A9000DFDDDBD9D7D5D3D1CFCFCBC9C7C5C3C124
:103AA000BFBDBBB9B7B5B3B1AFAFABA9A7A5A3A114
:103AB0009F9D9B99979593918F8F8B898785838104
:103AC0007F7D7B79777573716F6F6B6967656361F4
:103AD0005F5D5B59575553514F4F4B4947454341E4
:103AE0003F3D3B39373533312F2F2B2927252321D4
:103AF0001F1D1B19171513110F0F0B0907050301C4
:103B000000000000000000000000000000000000B5
:103B100000000000000000000000000000000000A5
:103B20000000000000000000000000000000000095
:103B30000000000000000000000000000000000085
:103B40000000000000000000000000000000000075
:103B50000000000000000000000000000000000065
:103B60000000000000000000000000000000000055
:103B70000000000000000000000000000000000045
:103B8000FFFFFFFFFFFFFFFFFFFFFFFFFFFFFFFF45
:103B9000FFFFFFFFFFFFFFFFFFFFFFFFFFFFFFFF35
:103BA000FFFFFFFFFFFFFFFFFFFFFFFFFFFFFFFF25
:103BB000FFFFFFFFFFFFFFFFFFFFFFFFFFFFFFFF15
:103BC000FFFFFFFFFFFFFFFFFFFFFFFFFFFFFFFF05
:103BD000FFFFFFFFFFFFFFFFFFFFFFFFFFFFFFFFF5
:103BE000FFFFFFFFFFFFFFFFFFFFFFFFFFFFFFFFE5
:103BF000FFFFFFFFFFFFFFFFFFFFFFFFFFFFFFFFD5
:00000001FF
